:01000000FF00
:10F200000075B0FFE5B05404602FC390F1FD7400A9
:10F210009394FF700EC390F1FC74009394FF7003FD
:10F2200002010090F1FD740093F5F090F1FC740080
:10F2300093F58285F0837400737581D012F27DC2DC
:10F2400098D29990F1FB740093F5F0C394FF602776
:10F250007550FF7551FF85F05230980302F303D5C6
:10F2600050F730980302F303D551EE30980302F3C0
:10F2700003D552E502F20A3098FD02F30375985A5D
:10F2800075CBFF75CAFA75C834753300223099FD05
:10F29000E534C299F5990022E542C412F2B4E54280
:10F2A00012F2B4E543C412F2B4E54312F2B4753479
:10F2B00068518D22540FC0E0C3940A10D70924412D
:10F2C000F534518DD0E022D0E02430F534518D2238
:10F2D000C0337533FAE58954F04401F5897561004E
:10F2E000C28C758CB8758A02C28DD28C20980C3075
:10F2F0008DFAD533EB756101D03322C298859941DF
:10F30000D0332200209805C29902F3BCC298D2994A
:10F31000C3E599942A600302F3AA12F65A6035F500
:10F32000F0C39454701475343F12F28D7534541236
:10F33000F28D749312F28D02F3BCE5F0C39453C3C3
:10F3400075343F12F28D75345312F28D749212F2AD
:10F350008D02F3BC788086E0C39446603886E0C3B3
:10F360009447700261D6788086E0C39457602986FE
:10F37000E0C39452602586E0C39445602186E0C3D3
:10F380009453601D86E0C3944C601986E0C394508A
:10F39000601502F3AA02F3C102F45002F3F402F47E
:10F3A000D702F52302F61A02F58175343F12F28D69
:10F3B00075344312F28D75348212F28DC29802F2C6
:10F3C0004375344612F28D75345612F28D75349CA5
:10F3D00012F28D02F3BC0886830886827534475189
:10F3E0008D753400518D753447518D75A8007400AA
:10F3F0007302F3AA7881864408864590F1FF740071
:10F4000093C3540C940C7002812075342112F28D38
:10F4100075345212F28D7473F53412F28D02F3BC0E
:10F42000854483854582C3E58394F230D7DCC37479
:10F430000093F54675345212F28DC374522546F589
:10F44000F085463412F28D85F03412F28D02F3BC51
:10F450007881864408864508864690F1FF740093BB
:10F460005403C39403601675345712F28D753452E9
:10F4700012F28D24A9F53412F28D02F3BCC3E544D7
:10F4800094F230D7E2C375F65575F6AA75F6557540
:10F49000BF048544F48545F58546F675F7808544B7
:10F4A00083854582740093C3954670157534571251
:10F4B000F28D75340012F28D75345712F28D02F30D
:10F4C000BC75345712F28D75342112F28D2478F503
:10F4D0003412F28D02F3BC75F65575F6AA75F65521
:10F4E00075BF0475F783900000C374009394FF7098
:10F4F0001DA3C3E58394F070F075344512F28D7549
:10F50000340012F28D75344512F28D02F3BC75345D
:10F510004512F28D75342112F28D75344512F28D3B
:10F5200002F3BC78818644C3E54494F130D70EC31E
:10F5300090F1FF740093C3543094306016753453C7
:10F5400012F28D75345212F28D74A5F53412F28DCB
:10F5500002F3BC75F65575F6AA75F65575BF0485A8
:10F5600044F475F50075F78275345312F28D7534D5
:10F570000012F28D7453F53412F28D02F3BC02F6D0
:10F580000579807881864408864508866A90F1FF6F
:10F59000740093C354039403601875345012F28DB1
:10F5A00075345212F28D74502452F53412F28D02D9
:10F5B000F3BC08C3E54494F230D7DFC375F6557544
:10F5C000F6AA75F65575BF048544F48545F586465B
:10F5D0008546F675F780854483854582740093C31C
:10F5E00095467021080545E54570020544D56AC376
:0FF5F00075345012F28D75340012F28D7534504F
:10F5FF0012F28D02F3BC75345012F28D7534211254
:10F60F00F28D75347112F28D02F3BC75F65575F6E5
:10F61F00AA75F65575BF040000000075F7817534A3
:10F62F004C12F28D75340012F28D75344C12F28D2E
:10F63F0002F3BC75344C12F28D75340012F28D75D5
:10F64F00346D12F28D02F3BC74542275610051D0E7
:10F65F008561E070F385413785413B753A2A7880A3
:10F66F00E53A2541F53A51D08561E070DBA64108B6
:10F67F00C3E894CF60D2C3D537E6883C18883D18CD
:10F68F00883E18883F02F6B9F53875F0F5E538A4CD
:10F69F00F5F0C374D9953825F0C4F538A83FE6C402
:10F6AF00C39538C3C4F618B880F4A83DE6C3953A9D
:08F6BF00600374532274002261
:10FA0000C0E0C083C082C0D0C0BF90F1FF7400933B
:10FA100054039403600D7CF0D0BFD0D0D082D0834B
:10FA2000D0E022C3EF94F010D70D7C0FD0BFD0D020
:10FA3000D082D083D0E022EFC3944030D70EC37C75
:10FA40000FD0BFD0D0D082D083D0E02275F65575CC
:10FA5000F6AA75F65575BF048FF48EF58DF675F719
:10FA6000808F838E82740093FDC39D700D7C00D0C7
:10FA7000BFD0D0D082D083D0E0227CFFD0BFD0D006
:07FA8000D082D083D0E02208
:10FB0000C0E0C083C082C0D0C020C0BF90F1FF74ED
:10FB10000093543003030303C2D79403600F7CF0B7
:10FB2000D0BFD020D0D0D082D083D0E022EFC394F9
:10FB3000EF10D70F7C0FD0BFD020D0D0D082D08391
:10FB4000D0E022EFC3944030D710C37C0FD0BFD099
:10FB500020D0D0D082D083D0E02275F65575F6AA99
:10FB600075F65575BF048FF475F50075F7828F2013
:10FB7000052005208F83758200740093C394FF7065
:10FB800017A3C3E583952070F07C00D0BFD020D0B0
:10FB9000D0D082D083D0E0227CFFD0BFD020D0D084
:07FBA000D082D083D0E022E7
:00000001FF
